:06000000008074022BA633
:03000B0002215877
:0300130002203890
:03001B000222605E
:03002300022B4F5E
:10002B0032534D505445204D616368696E652020F5
:10003B00202863292031393936202020416C636F09
:10004B00726E204D63427269646520496E632E2087
:10005B0020200D534D505445204D616368696E65EA
:10006B00202020012056312E37310D00C2AF75D024
:10007B000075816B43B0FF4390FF75892175880430
:10008B00758DFD758BFDD28E7589237598D0787F14
:10009B00E4F6D8FD751800751E149000007400F07E
:1000AB00A3A883B820F974FF90E800F0901523F013
:1000BB00740F90E000F0901522F090E000E0F890C3
:1000CB00E800E05875A015781EF2D294D296120172
:1000DB0078902D3512022C902D4812022C122CCC1C
:1000EB00121ADF121AB7121E8E122CDA122CCC1225
:1000FB001EF3122CCC122CCC122CCCC294122CDA58
:10010B00D29475B80075A811D2AF751296D221C2D0
:10011B0015C23FD201302A02C20175816B300144F6
:10012B00C28C758A00754C00C204D246D28CD2A9FF
:10013B00902D3512022C902D4812022CC22712053D
:10014B0006302303120BBB3001121202C93004EE2E
:10015B00C204B2941207DD30010280E2C28CC2A944
:10016B00C246D2922022030214B50217119000004E
:10017B0075A0A07802E230E70BA3E583B405F6C2C5
:10018B00380201C9D2387A301201CA7A301201CA48
:10019B007A381201CA7A801201CA7A061201CA7A17
:1001AB000C1201CA7A011201CA7A401201CA7A5A98
:1001BB001201E97A401201CA12020BB45AC122C0D1
:1001CB00F030381775F00075A0A07802E230E70721
:1001DB0000D5F0F30201E67800EAF2D0F022C0F08D
:1001EB0030381A75F00075A0A07802E230E70700EE
:1001FB00D5F0F302020875A0A07801EAF2D0F02244
:10020B00C0F030381975F00075A0A07802E230E725
:10021B000700D5F0F302022975A0A07803E2D0F015
:10022B0022740093A312024AFA740093A32AFA12BF
:10023B0001CA740093A36006FA1201E980F42283C9
:10024B00227FBF93D37A851201CAE55175F0006006
:10025B000475F00A842430FA1201E9E5F02430FA2F
:10026B001201E97A3A1201E9E55275F00060047562
:10027B00F00A842430FA1201E9E5F02430FA120175
:10028B00E97A3A1201E9E55375F000600475F00A5A
:10029B00842430FA1201E9E5F02430FA1201E97AEC
:1002AB002E1201E9E55475F000600475F00A842400
:1002BB0030FA1201E9E5F02430FA1201E922303A62
:1002CB0008E56830E0031202ED303B08E56830E1E9
:1002DB0003120424303C08E56830E203120427C201
:1002EB003A22E562C39561F4B41200500302042371
:1002FB00A86275A01C74FEF2F5F075A01B7401F2D8
:10030B000875A01CE56AF225F0F5F075A01BE4F268
:10031B000875A01C7428F225F0F5F075A01BE4F20B
:10032B000875A01CE569F225F0F5F075A01BE4F249
:10033B000875A01CE551F225F0F5F075A01BE4F251
:10034B000875A01CE5F0C313F275A01B7401F2082D
:10035B0075A01C74FEF2F5F075A01B7401F2087504
:10036B00A01CE56AF225F0F5F075A01BE4F2087508
:10037B00A01C7428F225F0F5F075A01BE4F20875AB
:10038B00A01CE5692401F225F0F5F075A01BE4F241
:10039B000875A01CE552F225F0F5F075A01BE4F2F0
:1003AB000875A01CE5F0C313F275A01B7401F208CD
:1003BB0075A01C74FEF2F5F075A01B7401F20875A4
:1003CB00A01CE56AF225F0F5F075A01BE4F20875A8
:1003DB00A01C7428F225F0F5F075A01BE4F208754B
:1003EB00A01CE5692402F225F0F5F075A01BE4F2E0
:1003FB000875A01CE553F225F0F5F075A01BE4F28F
:10040B000875A01CE5F0C313F275A01B7401F2086C
:10041B0088629060057406F022C23B22E562C395A8
:10042B0061F4B40C005003020505A86275A01C749E
:10043B00FEF2F5F075A01B7401F20875A01CE56ABD
:10044B00F225F0F5F075A01BE4F20875A01C7428DA
:10045B00F225F0F5F075A01BE4F20875A01CE56918
:10046B002404F225F0F5F075A01BE4F20875A01C2E
:10047B00901563E0F225F0F5F075A01BE4F208751A
:10048B00A01CE5F0C313F275A01B7401F20875A054
:10049B001C74FEF2F5F075A01B7401F20875A01C1C
:1004AB00E56AF225F0F5F075A01BE4F20875A01CC7
:1004BB007428F225F0F5F075A01BE4F20875A01C6A
:1004CB00E5692405F225F0F5F075A01BE4F208753B
:1004DB00A01C901564E0F225F0F5F075A01BE4F27A
:1004EB000875A01CE5F0C313F275A01B7401F2088C
:1004FB0088629060057406F0C23C22E559655A602B
:10050B000812053420232180F2E56365646008122C
:10051B0006DA20231380F2E55F6560600B202D0562
:10052B0012072E80031226CE22202103020603750A
:10053B00A01EA959E3FA75A01DE3FB0559C239C2E8
:10054B0029BB0006EA20280F802BEA30E7259015FF
:10055B005CF0D228020602C228B4FE0DF51CF51D74
:10056B00751800751E14020602B480005015751D17
:10057B00008047D229AD1DBDFE03020591BD0003CE
:10058B000205E1020602BB0002801AF5F090155C31
:10059B00E0251CC313B5F005D223020602745512D5
:1005AB00148A020602851EA0A818F2251CF51C0849
:1005BB008818B80002051E02060290155CE07583D0
:1005CB001C856282F0740175831BF00582E5616501
:1005DB0082602485826220391E75831C856282EAC3
:1005EB00F0EB75831BF00582E561658260098582FE
:1005FB00629060057406F02275A01EA959E3FA05F6
:10060B0059C239C229BAF50CEA202816201D31200F
:10061B001C398044EA90155CF0C21DC21CD2280222
:10062B0006D9C228D21DB4FE0DF51CF51D75180098
:10063B00751E140206D9B48000502B751D00805C0A
:10064B00C21DD21C251CF51C0206D9C21CFB0B2596
:10065B001CF51C0206D9D229AD1DBDFE0302059166
:10066B00BD00030206BD0206D91BBB001AF5F090B4
:10067B00155CE0251CC313B5F005D2230206D97413
:10068B005512148A0206D9851EA0A818F2251CF54E
:10069B001C088818B80002051E0206D990155CE0EC
:1006AB0075831C856282F00582E5616582601F851A
:1006BB00826220391975831C856282EAF00582E516
:1006CB0061658260098582629060057406F0223054
:1006DB00212B75A01AA963E3FA75A019E3FB056337
:1006EB0075831F855C82EAF00582E55B658260039A
:1006FB0085825C202002D299D23902054A75A01A54
:10070B00A963E3FA056375831F855C82EAF00582B2
:10071B00E55B6582600385825C202002D299D23929
:10072B0002060E75A016A85FE2055FB4FE0BD23071
:10073B00C231C232C2330207DC30300AB41302D2E8
:10074B0031C2300207DC303110B42000505E9015FE
:10075B0063F0C231D2320207DC30320A901564F0FA
:10076B00C232D233806B30334BF87A11901563E081
:10077B002AFA901564E02A547FC398702F90156461
:10078B00E0F8901563E09015652582F582740035CD
:10079B0083F583E8F0D23C30E504D23480037566F0
:1007AB001E901522E054FDF090E000F0C231C232F1
:1007BB00C233801DC231C232C23375831F855C8246
:1007CB00F00582E55B6582600385825C202002D2A6
:1007DB00992290E800E0F890E000E058C0E075A0A6
:1007EB0015781EE2FAD0E0F26A5AFAEA541F604D0D
:1007FB0030E025D291C201201510200015C23F30E8
:10080B002210301F0D12193A8008103F028003127C
:10081B00193AC200C215802530E105202B02D20007
:10082B0030E304D201801630220E30E402D21530B0
:10083B00E20BD201D291800530E202D20122785133
:10084B00E608460846084660121208677002800BDD
:10085B001208F460067D16DDFE80F522900000E0A4
:10086B006026F975650030257D20267A7E107F0085
:10087B008E828F83E0B4FF02806CF5F07851E6B581
:10088B00F00280104060D902805C74082EFEEF34B9
:10089B0000FF80DCA3E0B4FF02804BF5F008E6B567
:1008AB00F0028004404080DEA3E0B4FF028037F505
:1008BB00F008E6B5F0028004402C80CAA3E0B4FF38
:1008CB00028023F5F008E6B5F0028004401880B6EC
:1008DB00E565B4000DA3AB82AC83901520EBF0A3C0
:1008EB00ECF0056580A0E56522901520E0FBA3E008
:1008FB00FCE565B4000302093B8B828C83E0FEA30D
:10090B00E0FFA3E0F9700302092AA3E0B4FF03029E
:10091B00093EB48000500302096DD565028011EBCE
:10092B002408FB901520F0A3EC3400FCF002090422
:10093B00E56522E55CC3955BF489F0B5F0005003E7
:10094B0002093B8E828F83A85C75A01FE0F2A3087F
:10095B00D9FA885C202002D299D5650302093B02A3
:10096B00092AE562C39561F489F0B5F000500302E2
:10097B00093B8E828F83A86275A01CE0D2E7F275CB
:10098B00A01B7401F2D903088022A308D902800F9F
:10099B00E075A01CF275A01B7400F2A308D9F1E05E
:1009AB0075A01CF275A01B7401F2A30888629060FD
:1009BB00057406F0D5650302093B02092AE538C424
:1009CB00540FF5F0E53954F045F030E72530E622C9
:1009DB00543FF5F0B43F028024900007E0B5F002DD
:1009EB00801B901500E0600AFAA3E0B5F002800DC1
:1009FB00DAF790153EE4F0A3F0A3F08008901536DB
:100A0B00E5F0F0D21622901536E0F5F0A3E53AC4E6
:100A1B00540FF9E53B543049F025F0F5F0A3E53CD4
:100A2B00C4540FF9E53D543049F025F0543FF5F02F
:100A3B00901536E5F0F022901536E0F5F0E53EC462
:100A4B00540FF9E53F543049B5F002800B90153E39
:100A5B00E4F0A3F0A3F08020C21E7903783E75A0CA
:100A6B0015E2F5F0E0B5F0028002D21EF2121D3B4A
:100A7B00D9EF301E03021D43227400B5520DB5533E
:100A8B000AB551077403B55400500122901526E0A6
:100A9B0060F9FA7400F0A3A85E121E87B40300403D
:100AAB00F875A018E0D2E7F2FB75A0177401F208F5
:100ABB0075A0187408F22BFB75A0177400F208755B
:100ACB00A018EBF275A0177400F208885E75A08071
:100ADB0079057406F3A3DAC1C21B22900000E07003
:100AEB0005D226020B3F75F000900005E0C395F090
:100AFB00900003F075F008900006E095F09000046C
:100B0B00F0900000E0C226C394025002802604FA43
:100B1B007505137504008504068505077907120B07
:100B2B00B1EAFB120B427907120BB1DBF679051216
:100B3B000BB1DAE2D22522C082C083A8058504A0BE
:100B4B00850782850683E0F5F0E2C395F0C0D012ED
:100B5B000B89E0F5F0E2D0D095F0C0D0120B89E014
:100B6B00F5F0E2D0D095F0C0D0120B89E0F5F0E2B1
:100B7B00D0D095F04003120B9DD083D08222C0E0E1
:100B8B001582E582B4FF02158318B8FF0215A0D0B9
:100B9B00E0227908E2F5F0E0F2E5F0F0A308B80006
:100BAB000205A0D9EF22E72408F719E73400F72252
:100BBB00901400E0B44203020E03543F2323900B26
:100BCB00CD73020CD500020EF300020F9400020F3E
:100BDB00A500020FC200020CCD00020FD000020FC5
:100BEB00F600021030000210BE0002129200021238
:100BFB00B6000212DC000212F6000213020002130E
:100C0B0052000213A9000214820002145E000214A7
:100C1B00380002140F0002104F0002106F00021276
:100C2B0026000213340002134100020CCD00020C0B
:100C3B00CD00020CCD00020CCD00020CCD00020C3D
:100C4B00CD00020CCD00020CCD00020CCD00020C2D
:100C5B00CD00020CCD00020CCD00020CCD00020C1D
:100C6B00CD00020CCD00020CCD00020CCD00020C0D
:100C7B00CD00020CCD00020CCD00020CCD00020CFD
:100C8B00CD00020CCD00020CCD00020CCD00020CED
:100C9B00CD00020CCD00020CCD00020CCD00020CDD
:100CAB00CD00020CCD00020CCD00020CCD00020CCD
:100CBB00CD00020CCD00020CCD00020CCD00020CBD
:100CCB00CD00745512148AC22322901401E0B4FE95
:100CDB0003020CF9B4FF03020D27B40003020D2726
:100CEB00B4FD03020D27745512148AC22322120D70
:100CFB000474AA12148AC223227A0790000074008B
:100D0B00F0A3DAFCD226D225751800751E14751FB8
:100D1B00007400900005F07408A3F022C21EF5F0D9
:100D2B00202606900000E07003020DF2FBF51F7AFF
:100D3B0001A9F0EA75F008A4240FF582E5F0340060
:100D4B00F58389F0E0B5F0028003020DE5D21EE5D4
:100D5B0082C39403F582E5839400F583E0FCA3E062
:100D6B00FDA3E0F9E51FC39A04C0F075F008A4AF2A
:100D7B00F0FEEA1475F008A42410F8E5F03400F541
:100D8B00A0EA75F008A42410F582E5F03400F58391
:100D9B00120E2EECF8EDF5A0E92CF58274003DF562
:100DAB00837400C39582FE74149583FF120E2E90EC
:100DBB000003E0C399F0A3E09400F0A3E0C399F023
:100DCB00A3E09400F0120E3DD0F01B151FE51FB4ED
:100DDB000003020CF9BB000C800D0ABB000280075C
:100DEB00DB028003020D3C301E06E51F900000F075
:100DFB0074AA12148AC22322A85C90005E7900E9BF
:100E0B00936016B40102744175A01FF20908E8B58E
:100E1B005BED2020FAD29980F6885C202002D299D3
:100E2B00C22322E0F2121D3BDEF9BF00028002DF7B
:100E3B00F222900014E51F6029F8E0C39CAE82AF4C
:100E4B0083A3E09505400D8E828F83E0C399F0A3B9
:100E5B00E09400F074072582F58274003583F583E6
:100E6B00D8D822900000E0F5F0FA7B007E0D9000C0
:100E7B0003E02AFA74003BFBA3DEF6900010AEF001
:100E8B00BE0003020E9F7F08E02AFA74003BFBA30F
:100E9B00DFF6DEF2900003E0FFA3E0FE900800EE29
:100EAB004F600FE02AFA74003BFBA31FBFFFF01E3D
:100EBB0080ED7E0F901500E02AFA74003BFBA3DE59
:100ECB00F67E0F90150FE02AFA74003BFBA3DEF6BB
:100EDB007E20901546E02AFA74003BFBA3DEF690C9
:100EEB000001EAF0A3EBF022900000E004B4FE084E
:100EFB00745512148A020F91F014F5F07408A4249F
:100F0B0010F8E5F03400F5A07A04901401E0F21229
:100F1B001D3BDAF9E0B4FE0E900000E014F07455BE
:100F2B0012148A020F91FDA3E0FCA3A982AA83905D
:100F3B000003E02CF0A3E03400F0900005E0F5F0A6
:100F4B00F2121D3BE0F2FB121D3BECF2121D3BEDCE
:100F5B00F2121D3B74FFF2121D3BF2121D3BF212FB
:100F6B001D3BF28A838982A9F0E08BA0F3A309B918
:100F7B0000010BDCF4900005E9F0A3EBF0C226C2F4
:100F8B002574AA12148AC2232220260620250312B6
:100F9B000AE674AA12148AC22322121CB074AA1273
:100FAB00148AC22320340B901522E04402F090E007
:100FBB0000F0D297D29622121ADF121EF374AA12E5
:100FCB00148AC22322901401E0B440004002801323
:100FDB00B40A00400E900007F0121CB074AA121451
:100FEB008A8005745512148AC22322901401E0B42E
:100FFB000A0040028022FA780075A015F2121D3B00
:10100B00E0B43F005012B43200400DF2DAEF74AA94
:10101B0012148A121CB0800A901500E4F074551259
:10102B00148AC22322780175A0149015467D20E204
:10103B00F0121D3BDDF9121CB0121EF374AA121430
:10104B008AC2232290155CE0547FF56A901401E06C
:10105B005407F568901402E0B41B004002741AF5B3
:10106B0069C22322900009E075F01E700375F01819
:10107B00B4010375F019901401E0B418004001E4B9
:10108B00901585F0901402E0B43C004001E49015FB
:10109B0086F0901403E0B43C004001E4901587F017
:1010AB00901404E0B5F0004001E4901588F0D23DB7
:1010BB00C22322901401E0700575F0188060B40112
:1010CB000575F0198058B4020575F01E8050B403F5
:1010DB000575F01E8048B4040575F01E804074023F
:1010EB00900009F090150F7400F0A37400F0A37436
:1010FB0000F0A37400F0A37418F0A37400F0A374B1
:10110B0000F0A37400F0A37400F0A37400F0A374B8
:10111B0000F0A37400F0745512148A02121A900096
:10112B0009F0901402E0B4180050B390150FF0F5CD
:10113B0055901517F0901403E0B43C0050A0901597
:10114B0010F0F556901518F0901404E0B43C0050D4
:10115B008D901511F0F557901519F0901405E0B519
:10116B00F00040030210E9901512F0F55890151A93
:10117B00F0C223901406E0B41804D2238005400378
:10118B000210E9901513F0F530901407E0B43C0011
:10119B0040030210E930230560030210E990151497
:1011AB00F0F531901408E0B43C0040030210E93034
:1011BB00230560030210E9901515F0F53290140920
:1011CB00E0B5F00040030210E93023056003021084
:1011DB00E9901516F0F53390140AE0A2E09222A2E2
:1011EB00E19205A2E2921FA2E3922AA2E4922BA221
:1011FB00E5922DA2E6922EA2E79213900008F0D270
:10120B0096202204C2018002D20174AA12148A12FF
:10121B001CB0121EF3121E8EC22322900009E07521
:10122B00F01E700375F018B4010375F019901401DA
:10123B00E0B4180040028047901402E0B43C004038
:10124B0002803C901403E0B43C00400280319014C7
:10125B0004E0B5F0004002802690151AF0901403BC
:10126B00E0901519F0901402E0901518F09014010D
:10127B00E0901517F074AA12148A121CB080057432
:10128B005512148AC22322901401E0FBA3E0FA90BA
:10129B001522E04AF0FAA3E04BF090E800F090E062
:1012AB0000EAF074AA12148AC22322901401E0F40B
:1012BB00FBA3E0F4FA901522E05AF0FAA3E05BF0FE
:1012CB0090E800F090E000EAF074AA12148AC223AE
:1012DB002290E800E0FB90E000E0FA74AA12148A76
:1012EB00EB12148AEA12148AC22322D201D291740D
:1012FB00AA12148AC22322D29120151720001CC2D5
:10130B003F302217301F14300304D201801A1219F8
:10131B003A8008103F02800312193AC201C200C280
:10132B001574AA12148AC22322202B02D20074AA8B
:10133B0012148AC22322302206C2AFD215D2AF7446
:10134B00AA12148AC22322901401E0A2E090000892
:10135B00E092E35000F075A015781B901402E0F9B1
:10136B00F208A3E0FAF208A3E0F2FBC3740099744D
:10137B008D9A74279B400302139E900008E054F74C
:10138B00F090151B7400F0A3F0A3F0745512148A9F
:10139B000213A6121CB074AA12148AC22322900044
:1013AB0000E0FFFA12148A9000100FDF02804EE06B
:1013BB0012148A2AFAA3E012148A2AFAA3E012144E
:1013CB008A2AFAA3E012148A2AFAA3E0FDA3E0FE0C
:1013DB00A3E0FCA3E0A312148A2AFAEC12148A2AC3
:1013EB00FAC082C0838D828E830CDC028009E012EE
:1013FB00148A2AFAA380F3D083D08280AEEA121427
:10140B008AC223227F037E007A00903400E01214FC
:10141B008A2AFAA3DEF7DFF59020007E10E0121483
:10142B008A2AFAA3DEF7EA12148AC22322901565E0
:10143B007F20E4F0A3DFFC756600C234C235C236F0
:10144B00901522E04402F090E000F074AA12148A86
:10145B00C22322E430350244013036024402FA1230
:10146B00148A9015657F20E012148A2AFAA3DFF7FD
:10147B00EA12148AC2232274AA12148AC22322C02B
:10148B00E0C082C08375831F855C82F0E55C04F548
:10149B0083B55B072020FAD29980F685835C2020E8
:1014AB0002D299D083D082D0E02275A891C28CC28F
:1014BB008EC28F902D5B12022C902D6B12022C90F2
:1014CB002D9312022CC20BC20DC212C20FC20CC240
:1014DB0010C20EC207851211758A00754C00752952
:1014EB0040752A01755500755600755700755800E3
:1014FB0075330090151BE0F530A3E0F531A3E0F553
:10150B0032C2AF75B80675A81FD246D28CD2AFC205
:10151B0023121AB712050630230D75A891C28CC27F
:10152B008E120BBB0216FC100C183004E7C204120F
:10153B0002C91207DD3001DC75A891C28CC28E0284
:10154B0016FCE539540375F00AA4F8E538540F2856
:10155B00200E09B415BED20E7A0080B8F890157023
:10156B00EA540323738006800A800E8028B8166F16
:10157B000A80A1B817690A809BB818030A8095B82E
:10158B00005D75461875127875295BC206902DE3C0
:10159B0012022C804FB8193175461E75129675299B
:1015AB0015C206E53930E20AD206902DFE12022C46
:1015BB008032900009E0B40208902DF512022C80C5
:1015CB0023902E0712022C801BB800137546197539
:1015DB00127D75294DC206902DEC12022C8005C28E
:1015EB000E02151F902D7912022CC2AF8543418537
:1015FB004442D2AFE54175F014A4F541A8F0E542A1
:10160B0075F014A428F542754E00754D00D210D21A
:10161B000FE539540375F00AA4F5F0E538540F259E
:10162B00F004F548F554E53B540775F00AA4F5F0C2
:10163B00E53A540F25F0F549F553E53D540775F0A0
:10164B000AA4F5F0E53C540F25F0F54AF552E53FB9
:10165B00540375F00AA4F5F0E53E540F25F0F54B55
:10166B00F551D23A121AB7C202C218C219120506A4
:10167B0030230302152520100D75A891C28CC28E44
:10168B007528000216FC301902C219301836C21820
:10169B001207DD30010975A891C28CC28E805230C1
:1016AB000D0B1209C8902D7912022C8017902D86E4
:1016BB0012022CD296E511600BD51108D236C2015D
:1016CB00C222802D30021AC202301603120A1130C8
:1016DB001B03120A84120849121F7C1202C9120240
:1016EB005030170AC217301605C216120A420216DC
:1016FB0078121AB7D297D296901522E04409F0903F
:10170B00E000F002012575A891C28CC28EC215C2F1
:10171B003FC21AC218901522E054FEF090E000F080
:10172B00902D6312022C12193A20426420413A2068
:10173B004025754618754000901554E0B4E90C909F
:10174B002DE312022C9015540217AE902DDA1202D3
:10175B002C9015540217AE902DEC12022C901556AE
:10176B007546197540000217AE304012902DF512D8
:10177B00022C90155A75461E7540000217AE902D1F
:10178B00FE12022C90155875461E7540040217AEBA
:10179B00902E0712022C90155875461E754000C2EC
:1017AB0040C241E0A3750F00F50EE0F50D75470043
:1017BB00750936750C00750B0A750A01D209850E71
:1017CB004F121AB7C2AF75B802850E8A202E13902E
:1017DB002DB3202703902DA612022C75A81BD28C9B
:1017EB00805775A81FC28B902D6B12022C902DCD9C
:1017FB0012022C20412F204016902DDA12022C744D
:10180B00EA750F00F50E850E4F74C2F50D802A9008
:10181B002DEC12022C750F0074E0F50E850E4F7433
:10182B0097F50D801474BA750F00F50E850E4F7475
:10183B00F0F50D902E0712022CC246C28DC28FD22C
:10184B00AFC2231224C7D203120506302306120B94
:10185B00BB200167302714901589E0B4050C902D3F
:10186B00A612022CD297C2278001F030240FE54537
:10187B00B40302800875450312251980CB3002167C
:10188B00754500122519C224C2021208497545017B
:10189B0012251912025030181C754502122519C257
:1018AB00181207DD121F7C20011130150B902DC073
:1018BB0012022C801202185302185375A891C28C75
:1018CB00C28E752800805612050620233030022563
:1018DB00C2021202C91207DD200136201517D2925F
:1018EB00202E09902DA612022C021853902DCD12EA
:1018FB00022C0218533018CFC2180218D2120BBB8D
:10190B003015DBD29175A891C28CC28E75280080E0
:10191B000CD29175A891C28CC28E7528009015229D
:10192B00E04401F090E000F0D296C20302012512D0
:10193B001AB790150FE0F555A3E0F556A3E0F55750
:10194B00A3E0F558A3E0F530A3E0F531A3E0F532C1
:10195B00A3E0F533A330000390150FE0F54BA3E0A4
:10196B00F54AA3E0F549A3E0F548303D1290158503
:10197B00E0F54BA3E0F54AA3E0F549A3E0F5489069
:10198B000009E070087528007567048027B401080A
:10199B00752801756704801CB403087528047567E6
:1019AB00018011B40408752802756701800675283B
:1019BB00037567017536FC7537BFE54875F00A840A
:1019CB0085F0384540F539E54975F00A8485F03ADC
:1019DB00F53BE54A75F00A8485F03CF53DE54B7522
:1019EB00F00A8485F03EF53F2290400374C2C2AFEB
:1019FB00F0904000E0E0F4FCE0F4FD90400374361E
:101A0B00F0904000E4F0F0D2AF202C43ED13547F64
:101A1B00FDEC132403FCED3400FDC3E5349CFC907A
:101A2B006003F0E5359DFD906003F075F00030E745
:101A3B000375F0FFAEF0C390155EE03CFCF0A3E045
:101A4B003DFDF0A3E03EFEF020E70C4D4C702EC2A6
:101A5B002CAD2CAC2D804775F00AF47013EDF4709F
:101A6B000FECF4B45000500803030303540FF5F0CC
:101A7B00E52CC395F0FDE52D9400FC802175F00A53
:101A8B00EE7011ED700EECB450005008030303031D
:101A9B00540FF5F0E52C25F0FDE52D3400FC75A079
:101AAB00407801EDC2AFF2ECF2D2AF22D22CE4902F
:101ABB00155EF0A3F0A3F0AD2CAC2D121AA9227A6F
:101ACB00108003121D3BE2F0DAF9FAE0C39A70FBC7
:101ADB00121D3B22120D04121C67903440E0B455CA
:101AEB000D902000E0FCB4FE004006021B8C021B94
:101AFB00DF902003E0A3F8C3740098E0F8740C980F
:101B0B005003021B8C90200075A0007800ECF27D36
:101B1B0000FE121D3BE0FBF2121D3BE0FAF2121D20
:101B2B003B7F0DE0F22CFC74003DFD121D3BDFF3FF
:101B3B00BE0004D226804AC226902010781075A0D1
:101B4B00007F08E0F22CFC74003DFD121D3BDFF31F
:101B5B00DEEF7E08E0F2121D3BDEF9900003E0FFA2
:101B6B00A3E0FE90280075A0087800EE4F6012E00D
:101B7B00F2121D3B2CFC74003DFD1FBFFFED1E80C0
:101B8B00EA7F0F780075A015903400E0F2121D3B30
:101B9B002CFC74003DFDDFF37F0F780F75A01590C3
:101BAB003410E0F2121D3B2CFC74003DFDDFF37F83
:101BBB0020784675A015903420E0F2121D3B2CFCCA
:101BCB0074003DFDDFF3ED8AF0B5F008EC8BF0B55A
:101BDB00F0028030901522E054FDF090E000F0D23E
:101BEB0035C297C296122CCC122CCCD297D2967CA3
:101BFB00209034FF7A107400A3F0DAFCE0B400FC00
:101C0B00DCF28010900000E06006C226D225800432
:101C1B00D226C2257D04785590150FE0F6A308DD7A
:101C2B00FA7D047830901513E0F6A308DDFA9000E6
:101C3B0008E0A2E09222A2E19205A2E2921FA2E3A7
:101C4B00922AA2E4922BA2E5922DA2E6922EA2E773
:101C5B009213202204C2018002D20122902CF5752E
:101C6B00A00078007A10E493F2121D3BDAF8902D65
:101C7B000575A01578007A0FE493F2121D3BDAF884
:101C8B00902D2675A015780F7A0FE493F2121D3B59
:101C9B00DAF8902D1075A01578467A16E493F212A7
:101CAB001D3BDAF822202606202503120AE6120E27
:101CBB006E780075A000902000E2FC121ACAEC703E
:101CCB0003021D04C31304FC121ACADCFB900003AD
:101CDB00E0FCFFA3E0FD7A04EDC313FDEC13FCDA8B
:101CEB00F7EF540F60010CBC0002800D780075A05B
:101CFB0008902800121ACADCFB780075A0159034E6
:101D0B0000121ACA780F75A015903410121ACA78DF
:101D1B004675A015903420121ACA785675A01590E6
:101D2B003430121ACA9034407455F0E0B455FC228A
:101D3B00A308B8000205A022901537E0540F232307
:101D4B00901D4F73021D8F00021D8F00021D8F000F
:101D5B00021D8F00021D9000021D9C00021DA80099
:101D6B00021DB400021E1D00021E3700021E510090
:101D7B00021E6C00021D8F00021D8F00021D8F00C2
:101D8B00021D8F0022901538E0543FFA7918021D7E
:101D9B00C0901538E0543FFA7919021DC0901538E0
:101DAB00E0543FFA791A021DC0901538E0543FFAFF
:101DBB00791B021DC0E562C39561F4B405005002A6
:101DCB0080F375831C75A01B85628274FF4480FBB6
:101DDB00F07401A882F205827400F02BFB7400A84A
:101DEB0082F20582E9547FF02BFB7400A882F20586
:101DFB0082EAF02BFB7400A882F20582EB03547F7E
:101E0B00F07401A882F205828582629060057406E7
:101E1B00F022901537E0232354C0F9A3E0543F4937
:101E2B00F9901522E049F090E000F022901537E090
:101E3B00232354C0F9A3E0543F49F9901523E049FB
:101E4B00F090E800F022901537E0232354C0F9A35B
:101E5B00E0543F49F4F9901522E059F090E000F07E
:101E6B0022901537E0232354C0F9A3E0543F49F4E3
:101E7B00F9901523E059F090E800F022E55EC39548
:101E8B005DF4229060027415F0906000741BF07486
:101E9B0007F0A374BBF09060047408F090600274B8
:101EAB0005F090600274B5F09060057406F09080B8
:101EBB00027415F0908000202D04741B80027413A3
:101ECB00F07407F0A3202D0474BB800274CCF09047
:101EDB0080047408F09080027405F090800274B551
:101EEB00F09080057406F022121AB7901546E0F5B3
:101EFB002B6000A3A3A3E0F52DA3E0C0E054FEC329
:101F0B009432F52CE52D9400F52D9040037476F06A
:101F1B009040017F32E52C2402F52CF0E52D3400A6
:101F2B00F52DF0122CECDFED7F19E52CC39402F5A7
:101F3B002CF0E52D9400F52DF0122CECDFECD0E01D
:101F4B00F52CF0E52DF0121F5522900009E0B4009E
:101F5B000590154C8013B4010590154E800BB402FF
:101F6B00059015528003901550E0F535A3E0F5343C
:101F7B0022C0D0C0E0C0F0C082C083202D0E301331
:101F8B000BE562C39562F4B40800500302202D7573
:101F9B00831C85628274FEF0F5F075831B7401F06F
:101FAB00058275831C7400F025F0F5F075831BE436
:101FBB00F0058275831C7460F025F0F5F075831BBA
:101FCB00E4F0058275831CE54BF025F0F5F0758385
:101FDB001BE4F0058275831CE54AF025F0F5F075DE
:101FEB00831BE4F0058275831CE549F025F0F5F0C1
:101FFB0075831BE4F0058275831CE548F025F0F52D
:10200B00F075831BE4F0058275831CE5F003547FA8
:10201B00F075831B7401F0058285826290600574F4
:10202B0006F0D083D082D0F0D0E0D0D0222046036F
:10203B00D28C32C0D0C0E0D214300D02B2967402F2
:10204B00C28CC58AD28CF54FE4C54C308D07047019
:10205B00027403C28DF550C3E54F948AE55094008A
:10206B00401BC3E529954FE52A95504004D20880C3
:10207B001374B5954F74029550C2085007C20BC22A
:10208B000D02215330080D30070A200A28C207051C
:10209B0047022153200B6BA208E53713F537E536C2
:1020AB0013F536B4FC78E537B4BF73300807D20AA2
:1020BB00D207022153C294D2177400B54808B54910
:1020CB0005B54A028016E53F540775F00AA4F5F0F2
:1020DB00E53E540F25F0F54BF551D23A750938759D
:1020EB000B08750A08754700D20BC20AC207300FDE
:1020FB0057754500754E00754D00D28ED28FC20FAD
:10210B008046C000A208A809E613F6D000D50A0E37
:10211B000509750A08D50B06C20BD20DD20C300877
:10212B0004D20780230547C207E54354F02544C476
:10213B00F50FE54F54F02550C4254350020544C319
:10214B00950FF54350021544D0E0D0D03220460312
:10215B0002216EC0E0054CE54C7005D204754C03B2
:10216B00D0E032C0D0C0E0C0F0C082C083300911D3
:10217B00301507300504D2968002B296C2070222B0
:10218B001FC000A809E630E00E301507300504D259
:10219B00968002B296D20703F6D0000547E50AC334
:1021AB0033F50A506F750A010509D50B67750936AA
:1021BB00750B0A754700854854854953854A5285E6
:1021CB004B51D23AE54875F00A8485F0384540F515
:1021DB0039E54975F00A8485F03AF53BE54A75F027
:1021EB000A8485F03CF53DE54B75F00A8485F03E9D
:1021FB00F53FD28F302E1DD5671AB209050CC28C54
:10220B00758AFE756701E5285407B40200503B75CB
:10221B0067048036B209850E4FE50CC3950D40025D
:10222B00054F050CC28CE4C3954F258AF58AD28CD9
:10223B00201A0DE509B43B12D21AD218D294800A97
:10224B00202407E509B43E02D224D083D082D0F0FB
:10225B00D0E0D0D0322046030225F5C0D0C0E0E557
:10226B004E6004154E8019E54D601AC3E4954D750B
:10227B004D00C28E258C5004D28E8009F58CD28EE7
:10228B00D0E0D0D032122519C21AE5457007200DC7
:10229B000DC2948009B40206D21AD294D218C0F09F
:1022AB00C083C082200D030223EA201A0C101406EF
:1022BB00C20DC20BD20F0223EA53A8FB854C178524
:1022CB008A16E547A20785441485431543A8049253
:1022DB0011F5F0B428004003022368C3742895F06D
:1022EB0023F5139415400BC20DC212C20BD20F0271
:1022FB0023EAE514C313C51513F51420110BC3956D
:10230B0016E5159517400280021513E5148513F099
:10231B00A4F51685F017E5158513F0A42517C3133F
:10232B00C51613C516C313F517E51613F516E517E2
:10233B00C313F515E51613C515C313C51513F514FE
:10234B002541F541E5153542F542E5162541F54D9B
:10235B00E5173542F54E154ED2120223F29428237F
:10236B00F5139415400BC20DC212C20BD20F0223F0
:10237B00EAE514C313C51513F51420110BC39516F9
:10238B00E5159517400280020513E5148513F0A49B
:10239B00F51685F017E5158513F0A42517C313C59E
:1023AB001613C516C313F517E51613F516E517C364
:1023BB0013F515E51613C515C313C51513F514C37E
:1023CB00E5419514F541E5429515F542C3E5419577
:1023DB0016F54DE5429517F54E154ED21280088530
:1023EB00424E85414D154EE545B403028008B401BC
:1023FB0002D2190224B7300D58301255C2979015DE
:10240B0022E054F6F090E000F0851211E539540308
:10241B0075F00AA4F5F0E538540F25F0F548E53BC7
:10242B00540775F00AA4F5F0E53A540F25F0F54979
:10243B00E53D540775F00AA4F5F0E53C540F25F083
:10244B00F54A7400B5481AB54917B54A14054880C2
:10245B004BD297901522E04408F090E000F0121A4E
:10246B00B70548E548B546347548000549E549B414
:10247B003C2A754900054A300610E54A75F00A8476
:10248B00E5F0600674022548F548E54AB43C0D7545
:10249B004A00054BE54BB41803754B008548548532
:1024AB004953854A52854B51D202D23A0545534581
:1024BB0003D082D083D0F0D0E0D0D032302D4E304C
:1024CB00134B74F012291B747F12291B747F122972
:1024DB001B740112291B740112291B900009E0B413
:1024EB0000028010B4010474208009B402047460EB
:1024FB0080027440454B12291BE54A12291BE54902
:10250B0012291BE54812291B74F712291B22302DA7
:10251B001930131620375CE545B4001174F11229FC
:10252B001BE548540F440012291B0225F4B4011576
:10253B0074F112291BE54854F075F0108444101205
:10254B00291B0225F4B4021174F112291BE549541D
:10255B000F442012291B0225F4B4031474F1122921
:10256B001BE54954F075F01084443012291BD23707
:10257B000225F4E545B4001174F112291BE54A5408
:10258B000F444012291B0225F4B4011574F11229D2
:10259B001BE54A54F075F01084445012291B022598
:1025AB00F4B4021174F112291BE54B540F44601261
:1025BB00291B0225F4B4033174F112291BE54B548A
:1025CB00F075F01084F5F0900009E0B40002801073
:1025DB00B4010474028009B402047406800274040A
:1025EB0045F0447012291BC23722C0D0C0E0C0F0A6
:1025FB00C083C0823015030226BD203D4390158950
:10260B00E004F00548E548B5464D7548000549E539
:10261B0049B43C43754900054A30411020400DE553
:10262B004A75F00A84C5F06003754802E54AB43C6C
:10263B0026754A00054BE54BB4181C754B008017EB
:10264B00901585E0F54BA3E0F54AA3E0F549A3E02F
:10265B00F548C23D20275BE54BB53056E54AB53111
:10266B0051E549B5324CE548B53347D291302B2370
:10267B00200511D215D23F901522E04401F090E0D5
:10268B0000F0802ED201901522E04401F090E00082
:10269B00F0801F3000102005EB901522E04401F074
:1026AB0090E000F080CD85554B85564A855749857E
:1026BB005848D202C21AC294D082D083D0F0D0E054
:1026CB00D0D032E560C3955F855F1BB40700500324
:1026DB000229D1122B45B4F1030229D5B4F06B12A8
:1026EB002B4520E763B47F62122B4520E75AB47F5A
:1026FB0002800B2409F5F0900007E0B5F04C122B8B
:10270B004520E744B402028006B4013E02281912A8
:10271B002B4520E733B410028008B430028003B499
:10272B007F28122B4520E720F51AB415030228B693
:10273B00B416030228B6B417030228B6B418030262
:10274B0028B6B41905022758151B0229CBE560C31F
:10275B00955FB4120050030229D1122B4520E7E8F4
:10276B00C3943075F00AA4F5F0122B4520E7D9C3BA
:10277B00943025F0B418004001E4901585F0122B2D
:10278B004520E7C4B400C3122B4520E7BBC39430EC
:10279B0075F00AA4F5F0122B4520E7ACC394302555
:1027AB00F0B43C004001E4901586F0122B4520E775
:1027BB0097B40096122B4520E78EC3943075F00A20
:1027CB00A4F5F0122B4520E73FC3943025F0B43C21
:1027DB00004001E4901587F0122B4520E72AB40046
:1027EB002A122B4520E721C3943075F00AA4F5F08B
:1027FB00122B4520E712C3943025F0B41F00400183
:10280B00E4901588F00228B6022753022755E5609D
:10281B00C3955FB40A0050030229D1122B4520E760
:10282B00E7C3B401E6122B4520E7DDC3F5F0540FE7
:10283B00B4180040030228B3901585F0E5F05460FE
:10284B0075F02084900009B4000474018010B40169
:10285B000474028009B40204740380027402122B04
:10286B004520E741C3B43C0040030228B3901586D2
:10287B00F0122B4520E72EC3B43C0040030228B3D3
:10288B00901587F0122B4520E71BC3B41F004003A4
:10289B000228B3901588F0122B4530E70BB4F705DF
:1028AB00D23D0229CB022753022755122B4530E785
:1028BB002CB4F72CE51AB4152AD291C201201510AD
:1028CB00200017C23F302212301F0F12193A800A14
:1028DB00103F02800512193AC2000229410229CB8E
:1028EB00022753B4160C3022F1C2AFD215D2AF026D
:1028FB002941B41705D201022941B41808202B0233
:10290B00D200022941B41905D23D0229410229CB3B
:10291B00C0E0758318855E82F07400758317F0052F
:10292B0082E55D6582600385825E9080057406F0AA
:10293B00851B5FD0E02274F0758318855E82F0747E
:10294B0000758317F00582E55D6582607385825E95
:10295B00747F758318855E82F07400758317F0059C
:10296B0082E55D6582605985825E74037583188587
:10297B005E82F07400758317F00582E55D658260F9
:10298B003F85825E7402758318855E82F0740075D4
:10299B008317F00582E55D6582602585825E74F79D
:1029AB00758318855E82F07400758317F00582E5D8
:1029BB005D6582600B85825E9080057406F08000F9
:1029CB00851B5F0226CE22022753122B4520E7F7E9
:1029DB00C0E054F075F01084540FB40018D0E054DC
:1029EB000FF5F090000AE054F045F0F090000EE087
:1029FB0014F00229CBB40116D0E0540F75F010A4DB
:102A0B00F5F090000AE0540F45F0F00229CBB40228
:102A1B0012D0E0540FF5F090000BE054F045F0F0BD
:102A2B000229CBB40316D0E0540F75F010A4F5F0C7
:102A3B0090000BE0540F45F0F00229CBB40412D0F8
:102A4B00E0540FF5F090000CE054F045F0F0022943
:102A5B00CBB40516D0E0540F75F010A4F5F0900030
:102A6B000CE0540F45F0F00229CBB40612D0E05421
:102A7B000FF5F090000DE054F045F0F00229CBB4C7
:102A8B00075DD0E0C0E0540175F010A4F5F09000A4
:102A9B000DE0540F45F0F0D0E0546075F0208490B9
:102AAB000009B4000990000EE004F0022AF5B4010D
:102ABB000990000EE004F0022AF5B4020B740390A7
:102ACB00000EE004F0022AF5B4030B740290000E22
:102ADB00E004F0022AF590000EE004F0022AF5D093
:102AEB00E090000EE0E4F00229CB90000EE0B40081
:102AFB004490000DE0901585F090000CE090158649
:102B0B00F090000BE0901587F090000AE09015888C
:102B1B00F090000FE0E4F0D23D901589E4F0200135
:102B2B001120270ED227C23FC215902DB312022CB3
:102B3B00C2970229CBE4F00229CB758316851B8241
:102B4B00E0051B22C0D0C0E0C082C08310990C10DE
:102B5B009826D083D082D0E0D0D032C299E55B6585
:102B6B005C7005C220022B80D220855B82055B75D1
:102B7B00831FE0F599022B57E59975831E855A82C1
:102B8B00F075831D209A04740080027401F0A3E594
:102B9B00596582600385825A022B57C0D0C0E0C0B2
:102BAB0082C083908005E030E103022C55908005B4
:102BBB00E030E203022CA0906005E030E103022B31
:102BCB00E1906005E030E205022C2980D6D083D05D
:102BDB0082D0E0D0D032E5616562700F90600574F1
:102BEB0004F090600274B5F0022BCC90600274A5D7
:102BFB00F09060027415F075831B856182E06008AC
:102C0B00906000741FF08006906000741BF0758359
:102C1B001C856182E0906003F00561022BCC906013
:102C2B0001E075831985648220E5047400800274C9
:102C3B0001F0906003E075831A856482F0A3E5636D
:102C4B0065826003858264022BD6E55D655E700F3D
:102C5B009080057404F090800274B5F0022BB8904C
:102C6B00800274A5F0202D1D9080027415F07583E1
:102C7B0017855D82E06008908000741FF0800690DD
:102C8B008000741BF0758318855D82E0908003F0E3
:102C9B00055D022BB8908001E0758317856082205B
:102CAB00E504740080027401F0908003E0758316D4
:102CBB00856082F0A3E55F65826003858260022BED
:102CCB00C27A3EEAC0E0122CDAD0E0FADAF5227AC8
:102CDB00007B20DAFEDBFC227A007B0ADAFEDBFCCF
:102CEB00227A007B32DAFEDBFC22000000000000BF
:102CFB00080A0202000000000000000000000000B3
:102D0B00000000000000000100040047C744E83940
:102D1B007B396CEE00E5CDBECEBD00000000001887
:102D2B0000000000000000008D27010120534D50D2
:102D3B005445204D616368696E65202000020120B7
:102D4B002056657273696F6E20312E37312020004B
:102D5B000101526561642000010147656E2020006E
:102D6B0001062D2D3A2D2D3A2D2D2E2D2D00020144
:102D7B004C6F636B65642020202000020153656C4F
:102D8B00662047656E2020000201417761697469F6
:102D9B006E6720534D505445202000020152756E32
:102DAB006E696E672020200002014D544320536C46
:102DBB006176652000020149646C696E67202020F2
:102DCB0020000201562D53796E6320202020000233
:102DDB000B32332E39373600020B323420667073C8
:102DEB0000020B32352066707300020B3330206605
:102DFB00707300020B32392E39376400020B3239F3
:052E0B002E39376E00B6
:00000001FF
